:1000000012C035C029C028C027C026C025C024C0C2
:1000100023C022C021C020C01FC01EC01DC01CC0E4
:100020001BC01AC019C011241FBECFEDCDBF10E0F8
:10003000A0E6B0E0E4E8F5E002C005900D92A0373C
:10004000B107D9F710E0A0E7B0E001C01D92A237D8
:10005000B107E1F770D094C2D3CFFC01808188232F
:1000600029F090E2919380818823E1F708951F920F
:100070000F920FB60F9211248F939F93EF93FF93DC
:100080008FE08A95F1F705B600FE27C0829B4AC033
:10009000E5E5F0E080818260808380818E7F8083CF
:1000A000839B0AC08091700090917100019790939A
:1000B00071008093700036C0849B05C0109271005F
:1000C000109270002FC08091700090917100019685
:1000D000909371008093700025C0829923C0E5E55C
:1000E000F0E0808183608083839B0AC080917000F0
:1000F000909171000196909371008093700012C0EE
:10010000849B07C08FEF9FE09093710080937000F5
:1001100009C08091700090917100019790937100D7
:1001200080937000FF91EF919F918F910F900FBE80
:100130000F901F901895CF92DF92EF92FF920F933E
:100140001F93DF93CF93CDB7DEB760970FB6F894C8
:10015000DEBF0FBECDBF188ACE0101967EDF8FE7CE
:1001600087BB11BA8CE182BBEBE5F0E08081806453
:1001700080838CE06FD136D1829B09C0E5E5F0E049
:1001800080818260808380818E7F808305C0E5E5E9
:10019000F0E080818360808378940F2EF0E6CF2E8C
:1001A000F0E0DF2EF02D8E010F5F1F4F0F2EFFEFBF
:1001B000EF2EFFE3FF2EF02D15D160E080E007D198
:1001C000C60128D161E080E002D180917000909159
:1001D00071004AE050E0B80190D1C8011BD1C701BD
:1001E0000197F1F7C80139DFE7CFE8E3F0E080815C
:1001F0008061808300C080818F7E808308951F93FB
:10020000982F662331F0E8E3F0E0808180648083FA
:1002100005C0E8E3F0E080818F7B8083A8E3B0E055
:100220008C918F7D8C93E7E3F0E080818860808300
:10023000808184608083808182608083808181600E
:1002400080838C918E7F8C938C918D7F8C938C91FD
:100250008B7F8C938C91877F8C9399232CF4E8E38C
:10026000F0E0808181608083192F96FF05C0E8E36C
:10027000F0E080818260808315FF05C0E8E3F0E054
:1002800080818460808314FF05C0E8E3F0E0808112
:1002900088608083AADFE8E3F0E080818E7F80833E
:1002A00080818D7F808380818B7F80838081877F29
:1002B000808313FF03C080818160808312FF05C0AB
:1002C000E8E3F0E080818260808311FF05C0E8E30D
:1002D000F0E080818460808310FF05C0E8E3F0E0F7
:1002E00080818860808381DFE8E3F0E0808188603E
:1002F000808380818460808380818260808380812C
:10030000816080831F910895882331F0E8E3F0E055
:1003100080818064808305C0E8E3F0E080818F7B8A
:100320008083A8E3B0E08C9180628C93E7E3F0E0F7
:100330008081877F808380818B7F808380818D7F98
:10034000808380818E7F80838C9180618C9300C0BC
:10035000B39B02C090E101C090E0B2999062B19964
:100360009064B0999068E8E3F0E080818F7E8083AC
:1003700000C080818061808300C0B3999160B29990
:100380009260B1999460B0999860E8E3F0E0808160
:100390008F7E8083892F089580E0B6DF8823E4F381
:1003A00088E090E00197F1F780E0AEDF08951F93B9
:1003B000182FF2DF60E0812F22DF1F9108951F9335
:1003C000182FEADF61E0812F1ADF1F91089566235D
:1003D00019F48058ECDF08958054E9DF0895DCDFDC
:1003E00090E0089581E0E3DF089582E0E0DF089582
:1003F0001F93182FD1DF1A3041F4803410F080E0C1
:1004000001C080E48058D3DF03C061E0812FF7DEB4
:100410001F910895CF93DF93FC018081882331F0F1
:10042000EF01E6DF898121968823D9F7DF91CF910B
:100430000895CF93DF93FC018491882341F0EF016D
:100440002196D6DFFE01219684918823D1F7DF9192
:10045000CF910895DF92EF92FF920F931F93D82EC2
:10046000E7E3F0E080818064808380818062808324
:1004700080818061808380818860808380818460C6
:10048000808380818260808380818160808380E03E
:100490009AEF0197F1F70F2EF8E3EF2EFF24F02DDE
:1004A000F7018081846080838081886080839DDE05
:1004B00080E09EE40197F1F798DE00E011E0C801CA
:1004C0000197F1F792DEC8010197F1F7F7018081FA
:1004D000877F80838ADEC8010197F1F788E267DFB2
:1004E00088E065DF7FDF86E062DF8D2D60DF1F91B2
:1004F0000F91FF90EF90DF900895FB019F01E8942A
:100500004230BCF04532ACF44A3029F497FB1EF47B
:10051000909581959F4F642F77271ED0805D8A33F9
:100520000CF0895D8193CB010097A9F716F45DE289
:1005300051931082C90100C0DC01FC01672F719149
:100540007723E1F7329704C07C916D9370836291B9
:10055000AE17BF07C8F30895AA1BBB1B51E107C024
:10056000AA1FBB1FA617B70710F0A61BB70B881F43
:10057000991F5A95A9F780959095BC01CD010895D2
:04058000F894FFCF1D
:10058400327820456E636F6465722064656D6F0018
:00000001FF
